:100000008A010B2849286428712877287C28B2287F
:10001000CD28272976290730831603139F009801DE
:100020001F3099008312980198178316071607103E
:1000300083120714C0308316810002206830F90053
:1000400007206530F90007206C30F90007206C307C
:10005000F90007206F30F90007200D30F900072064
:100060000A30F90007200130FB000820F300FF30C0
:100070007302031947280D307302031D442803201F
:100080000A30F900072047287308F40004203328B9
:1000900048288316831603130608C0398600831286
:1000A0000230F1000A203330F50005203230F5002F
:1000B00005202C30F50005200630F50005200C3019
:1000C000F5000520032008000130F500052001306F
:1000D000F1000A200230F50005200130F1000A206D
:1000E00008007408F6001030F700062008007508B4
:1000F000F600F701062008007608F000F00CF00C7E
:10010000F00C700C0F390F397704F80083120313C9
:100110000608C0397804F80086000130F1000A2092
:100120008312031386160130F1000A208312031391
:10013000861276080F397704F8000608C03978046B
:10014000F80086000130F1000A208312031386169E
:100150000130F1000A208312031386120130F100EE
:100160000A200800FA01831603139816043083123C
:10017000A3000920FA000C087A05003C031DC128E1
:10018000BB280708FF390319C6280130003C031DAE
:10019000CA28C128790899000800FC01FD01FE0168
:1001A000FF01FF3083120313A000A101A201071079
:1001B00055307B02031DDE280130A1001816A2086D
:1001C000031D02290530A3000920FC000C087C0552
:1001D000FF39003C0319EF280230A200DF28A108F4
:1001E000031D0129FB08031DF8280130A200012985
:1001F000FD03FD08031D0129FE03FE08031D01295F
:10020000FB03DF280230831203132202031D24297B
:100210000230A3000920FC0018087C05FF39003CCF
:10022000031915291A08FF0024290130A300092009
:10023000FC0018087C05FF39003C0319222918121C
:10024000181624291A08A000071420080800831291
:100250000313A4012308F0007008003C031D352996
:10026000013083120313A40074297008013C031D9C
:100270003E29023083120313A40074297008023C43
:10028000031D4729043083120313A4007429700846
:10029000033C031D5029083083120313A400742962
:1002A0007008043C031D5929103083120313A40065
:1002B00074297008053C031D622920308312031342
:1002C000A40074297008063C031D6B29403083127A
:1002D0000313A40074297008073C031D742980309F
:1002E00083120313A400742924080800DF30F200ED
:1002F00000000000000000000000000000000000FE
:1003000000000000000000000000000000000000ED
:1003100000000000000000000000000000000000DD
:0E032000F20B7D290000F10B76290000080089
:02400E003A3F37
:00000001FF
